:020000040000FA
:020000000528D1
:0800080000000030850000300B
:1000100086008316003085009F3081000030860006
:10002000831200308B001F2808003C309000900B9A
:100030001A28080064309100910B1C281728803082
:100040008600003085001420C03086000030850016
:100050001420E0308600003085001420F030860047
:10006000003085001420F830860000308500142010
:10007000FC308600003085001420FE308600003001
:1000800085001420FF3086000030850014201420E5
:100090000030860000308500142014208030860057
:1000A00000308500142001308600003085001420C7
:1000B00003308600003085001420073086000030B1
:1000C000850014200F3086000030850014201F307A
:1000D00086000030850014203F3086000030850007
:1000E00014207F308600003085001420FF30860009
:1000F000003085001420FF30860008308500142071
:10010000FF3086000C3085001420FF3086000E3052
:10011000850014201420FF3086000F308500142045
:100120001420003086000030850014200030860046
:10013000083085001420003086000C308500142023
:10014000003086000E3085001420003086000F300D
:1001500085001420803086000F3085001420813007
:1001600086000F3085001420833086000F30850014
:100170001420873086000F30850014208F308600D1
:100180000F30850014209F3086000F30850014202A
:10019000BF3086000F3085001420FF3086000F30FE
:1001A0008500142000308600003085001420FF30C8
:1001B00086000F3085001420003086000030850056
:1001C0001420FF3086000F30850014200030860098
:1001D000003085001420FF3086000F308500142089
:1001E0000030860000308500142014208030860006
:1001F0000030850014201420C030860000308500B7
:1002000014201420E03086000030850014201420D3
:10021000F03086000030850014201420F83086006D
:100220000030850014201420FC308600003085004A
:1002300014201420FE308600003085001420142085
:10024000FF308600003085001420FF308600083023
:1002500085001420FF3086000C3085001420FF300C
:1002600086000E3085001420FF3086000F30850098
:10027000142014201420003086000F308500142034
:1002800014201420AA3086000F308500142014207A
:100290001420553086000F308500142014201420BF
:1002A000AA30860000308500142014201420553018
:1002B00086000030850014201420142000308600B1
:1002C0000030850014201420C030860000308500E6
:1002D00014201420303086000030850014201420B3
:1002E0000C30860000308500142014200330860076
:1002F00000308500142014200C308600003085006A
:10030000142014200C3086000030850014201420A6
:10031000303086000030850014201420C030860064
:100320000030850014201420003086000030850045
:100330001420142014201420403086000030850042
:100340001420142050308600003085001420142022
:10035000543086000030850014201420553086006B
:100360000030850014201420D53086000030850030
:1003700014201420D530860000308500142014206D
:10038000D73086000030850014201420DF3086002E
:100390000030850014201420FF30860000308500D6
:1003A00014201420FF3086000F3085001420142004
:1003B0001420142014201420003086000030850002
:1003C00014201420013086000030850014201420F1
:1003D000053086000030850014201420153086007A
:1003E0000030850014201420553086000030850030
:1003F00014201420D53086000030850014201420ED
:10040000F53086000030850014201420FD30860071
:100410000030850014201420FF3086000030850055
:1004200014201420FF3086000F3085001420142083
:100430001420142000308600003085001420142081
:10044000003086000830850014201420003086001B
:100450000C30850014201420003086000E308500FA
:1004600014201420003086000F3085001420142042
:1004700000308600003085001420142000308600F3
:1004800001308500142014200030860003308500E0
:10049000142014200030860007308500142014201A
:1004A000003086000F3085001420142000308600B4
:1004B00000308500142014200030860001308500B3
:1004C00014201420003086000330850014201420EE
:1004D000003086000730850014201420003086008C
:1004E0000F30850014201420803086000F308500E6
:1004F00014201420C03086000F30850014201420F2
:10050000E03086000F30850014201420F030860083
:100510000F30850014201420F83086000F3085003D
:1005200014201420FC3086000F3085001420142085
:10053000FE3086000F30850014201420FF30860026
:100540000F30850014201420003086000030850014
:1005500014201420FF3086000F3085001420142052
:10056000FE3086000F30850014201420FC308600F9
:100570000F30850014201420F83086000F308500DD
:1005800014201420F03086000F3085001420142031
:10059000E03086000F30850014201420C030860023
:1005A0000F30850014201420803086000F30850025
:1005B00014201420003086000F30850014201420F1
:1005C000003086000E308500142014200030860094
:1005D0000C3085001420142000308600083085007F
:1005E00014201420003086000030850014201420D0
:1005F00014201420AA3086000A308500142014200C
:100600001420142055308600053085001420142055
:10061000142014200030860000308500142014209F
:06062000142014201F2825
:02400E00F33F7E
:00000001FF
